:1000000000308A00E7280000FF00030E8301A100F2
:100010007F08A0000A08A8008A01A00E0408A20018
:100020007708A3007808A4007908A5007A08A6003C
:100030007B08A700831383120B1E20288B183328FC
:10004000220884002308F7002408F8002508F90096
:100050002608FA002708FB0028088A00210E8300E2
:10006000FF0E7F0E09008A11352881018316861242
:10007000831286160108023C03183A282A08AE00AB
:10008000AE0803194828000000000000AE03402815
:10009000831686128312861201080A3C03184C2824
:1000A0008101291C92282910831601138B108312B9
:1000B0000B16C0308B048316061600308312061A06
:1000C0000130003A03195B280108AF0083160616B9
:1000D00000308312061A0130013C0319662801081A
:1000E000B0002F083002B1003108033C03188B2800
:1000F0003108073C031C8B281F151F197D281E087B
:10010000F700F70CF70C3F30F7057708A03CF80034
:100110002F087802AA000830F8001F08C7397804B1
:100120009F00CE282914831601178B1083120B16FB
:10013000C0308B048316061600308312061A013075
:10014000003A03199A280108AF00831606160030FA
:100150008312061A0130013C0319A5280108B000DA
:100160002F083002B1003108033C0318C8283108B9
:10017000073C031CC8281F151F19BC281E08F700C0
:10018000F70CF70C3F30F7057708203E2F07AA0041
:100190000030F8001F08C73978049F00CE288B1064
:1001A0008A1120282B30840000080319E62801302A
:1001B000F800F701F70BDA28F80BD9284A30F700D6
:1001C000F70BE02800000000800BD72800348401E2
:1001D0001F30830583161F129F121B0880399B0056
:1001E00007309C001F129F121B08803903389B00A8
:1001F0001F1383121F179F1783169F1383121F1439
:10020000941283160611861406120030831294008D
:10021000831694000108C0390738810083129001C9
:100220000030F800920000308316920007309C00E6
:1002300005080330F700F70B1B291C0883120D1368
:1002400083169D018F010F0864308312AB00D2200A
:100250000030F8001F08C73978049F000130AB0058
:10026000D22083160117831229141F151F1936294E
:100270001E08F700F70CF70C3F30F7057708203E13
:0C0280001E3EAA000B16C0308B04630069
:04400E00293FFC3F0B
:00000001FF
